:1000000010C02AC029C028C027C026C025C024C0CF
:1000100023C022C021C020C01FC01EC01DC01CC0E4
:100020001BC011241FBECFE5D2E0DEBFCDBF10E064
:10003000A0E6B0E0E8E2F2E003C0C89531960D9288
:10004000A036B107D1F710E0A0E6B0E001C01D92E4
:10005000A436B107E1F746C0D3CF9FEF97BB94BB5F
:1000600080EF8ABB91BB0895F92FE82F20E030E0A4
:100070008E2F9F2F64E670E0B9D02817390718F447
:100080002F5F3F4FF5CF0895C89B09C0C99B07C09C
:10009000CA9B05C0CB9B03C085E090E00895C89B38
:1000A00003C082E090E00895C99B03C084E090E023
:1000B0000895CA9B03C081E090E0089589B3992711
:1000C00023E0969587952A95E1F7282F392F2170FF
:1000D000307080FF03C083E090E00895932F822F5B
:1000E00008950895CFE5D2E0DEBFCDBFB6DFDC9A3C
:1000F0008EE190E0B9DFDC988EE190E0B5DFDC9A2C
:1001000081E0809363008093610080936000BCDF96
:10011000382FC817C1F1992783309105E9F0843051
:10012000910534F48130910549F0029769F02BC0B4
:1001300084309105B9F00597E9F025C080916300FE
:100140008F3108F58F5F05C0809163008823D9F057
:1001500081508093630017C0809161008F3198F4C3
:100160008F5F05C080916100882369F08150809382
:10017000610009C080916000843010F48F5F01C07D
:1001800081E0809360002091630028BB6091610052
:1001900065BB8091600099278230910571F08330B2
:1001A00091051CF4019739F013C08330910549F093
:1001B000049751F00DC0260F01C0261B209362004A
:1001C00007C0822F0AD002C0822F22D08093620003
:1001D0008091620082BBC32F9ACF002480FD060E5F
:1001E000660F11F08695D1F7802D089555270024CC
:1001F00080FF02C0060E571F660F771F611571053D
:1002000021F096958795009799F7952F802D089561
:10021000991B79E004C0991F961708F0961B881F58
:080220007A95C9F78095089555
:00000001FF
